 eglinfo

 Timestamp is 4be8c3e2 (Tue May 11 11:41:38 2010)

 Preferred load address is 00010000

 Start         Length     Name                   Class
 0001:00000000 00000004H .CRT$XCA                CODE
 0001:00000004 00000004H .CRT$XCZ                CODE
 0001:00000008 00000004H .CRT$XIA                CODE
 0001:0000000c 00000004H .CRT$XIZ                CODE
 0001:00000010 00000004H .CRT$XPA                CODE
 0001:00000014 00000004H .CRT$XPZ                CODE
 0001:00000018 00000004H .CRT$XTA                CODE
 0001:0000001c 00000004H .CRT$XTZ                CODE
 0001:00000020 00001868H .rdata                  CODE
 0001:00001888 00000024H .rdata$debug            CODE
 0001:000018ac 0000269cH .text                   CODE
 0001:00003f48 0000001cH .xdata                  CODE
 0001:00003f64 00000028H .idata$2                CODE
 0001:00003f8c 00000014H .idata$3                CODE
 0001:00003fa0 000000b4H .idata$4                CODE
 0001:00004054 00000018H .idata$6                CODE
 0001:0000406c 00000000H .edata                  CODE
 0002:00000000 000000b4H .idata$5                DATA
 0002:000000b4 00000008H .data                   DATA
 0002:000000bc 00000020H .bss                    DATA
 0003:00000000 000000e8H .pdata                  DATA

  Address         Publics by Value              Rva+Base       Lib:Object

 0000:00000000       ___safe_se_handler_table   00000000     <absolute>
 0000:00000000       ___safe_se_handler_count   00000000     <absolute>
 0001:00000000       __xc_a                     00011000     corelib0:crt0init.obj
 0001:00000004       __xc_z                     00011004     corelib0:crt0init.obj
 0001:00000008       __xi_a                     00011008     corelib0:crt0init.obj
 0001:0000000c       __xi_z                     0001100c     corelib0:crt0init.obj
 0001:00000010       __xp_a                     00011010     corelib0:crt0init.obj
 0001:00000014       __xp_z                     00011014     corelib0:crt0init.obj
 0001:00000018       __xt_a                     00011018     corelib0:crt0init.obj
 0001:0000001c       __xt_z                     0001101c     corelib0:crt0init.obj
 0001:0000003c       ??_C@_0BL@CHALDOEN@EGL_CONTEXT_CLIENT_VERSION?$AA@ 0001103c     eglinfo.obj
 0001:00000058       ??_C@_0BI@NHGJOHPG@EGL_CONTEXT_CLIENT_TYPE?$AA@ 00011058     eglinfo.obj
 0001:00000070       ??_C@_0BI@CIOBNPEL@EGL_VERTICAL_RESOLUTION?$AA@ 00011070     eglinfo.obj
 0001:00000088       ??_C@_0BD@HNDDKNFH@EGL_TEXTURE_TARGET?$AA@ 00011088     eglinfo.obj
 0001:0000009c       ??_C@_0BD@NPMMAJHI@EGL_TEXTURE_FORMAT?$AA@ 0001109c     eglinfo.obj
 0001:000000b0       ??_C@_0BC@NMADMDCO@EGL_SWAP_BEHAVIOR?$AA@ 000110b0     eglinfo.obj
 0001:000000c4       ??_C@_0BC@IBPIHKID@EGL_RENDER_BUFFER?$AA@ 000110c4     eglinfo.obj
 0001:000000d8       ??_C@_0BH@GMDOAKAE@EGL_PIXEL_ASPECT_RATIO?$AA@ 000110d8     eglinfo.obj
 0001:000000f0       ??_C@_0BB@JDFPHGGJ@EGL_MIPMAP_LEVEL?$AA@ 000110f0     eglinfo.obj
 0001:00000104       ??_C@_0BD@KKKDLOP@EGL_MIPMAP_TEXTURE?$AA@ 00011104     eglinfo.obj
 0001:00000118       ??_C@_0BE@CGCBKPDN@EGL_LARGEST_PBUFFER?$AA@ 00011118     eglinfo.obj
 0001:0000012c       ??_C@_0BK@CEHADGAI@EGL_HORIZONTAL_RESOLUTION?$AA@ 0001112c     eglinfo.obj
 0001:00000148       ??_C@_0L@CAKOEIEL@EGL_HEIGHT?$AA@ 00011148     eglinfo.obj
 0001:00000154       ??_C@_09HGLBPFCD@EGL_WIDTH?$AA@ 00011154     eglinfo.obj
 0001:00000160       ??_C@_0BC@ILOLBBKO@EGL_VG_COLORSPACE?$AA@ 00011160     eglinfo.obj
 0001:00000174       ??_C@_0BE@MAJLFKLF@EGL_VG_ALPHA_FORMAT?$AA@ 00011174     eglinfo.obj
 0001:00000188       ??_C@_0BL@ILCMOAGG@EGL_TRANSPARENT_BLUE_VALUE?$AA@ 00011188     eglinfo.obj
 0001:000001a4       ??_C@_0BM@JICEHDGJ@EGL_TRANSPARENT_GREEN_VALUE?$AA@ 000111a4     eglinfo.obj
 0001:000001c0       ??_C@_0BK@DCMMLEOK@EGL_TRANSPARENT_RED_VALUE?$AA@ 000111c0     eglinfo.obj
 0001:000001dc       ??_C@_0BF@GJLJHKPE@EGL_TRANSPARENT_TYPE?$AA@ 000111dc     eglinfo.obj
 0001:000001f4       ??_C@_0BB@ODEMPID@EGL_SURFACE_TYPE?$AA@ 000111f4     eglinfo.obj
 0001:00000208       ??_C@_0BB@MEILGNJE@EGL_STENCIL_SIZE?$AA@ 00011208     eglinfo.obj
 0001:0000021c       ??_C@_0M@HOPBGGDN@EGL_SAMPLES?$AA@ 0001121c     eglinfo.obj
 0001:00000228       ??_C@_0BD@EJBKGONN@EGL_SAMPLE_BUFFERS?$AA@ 00011228     eglinfo.obj
 0001:0000023c       ??_C@_0BE@IEOPKMAE@EGL_RENDERABLE_TYPE?$AA@ 0001123c     eglinfo.obj
 0001:00000250       ??_C@_0BH@MCJAMBFL@EGL_NATIVE_VISUAL_TYPE?$AA@ 00011250     eglinfo.obj
 0001:00000268       ??_C@_0BF@MMKMOGA@EGL_NATIVE_VISUAL_ID?$AA@ 00011268     eglinfo.obj
 0001:00000280       ??_C@_0BG@EMJKKPOL@EGL_NATIVE_RENDERABLE?$AA@ 00011280     eglinfo.obj
 0001:00000298       ??_C@_0BG@OCMLMIDO@EGL_MIN_SWAP_INTERVAL?$AA@ 00011298     eglinfo.obj
 0001:000002b0       ??_C@_0BG@LBGNNANK@EGL_MAX_SWAP_INTERVAL?$AA@ 000112b0     eglinfo.obj
 0001:000002c8       ??_C@_0BH@CHGKDLFB@EGL_MAX_PBUFFER_PIXELS?$AA@ 000112c8     eglinfo.obj
 0001:000002e0       ??_C@_0BH@LLFIGBCB@EGL_MAX_PBUFFER_HEIGHT?$AA@ 000112e0     eglinfo.obj
 0001:000002f8       ??_C@_0BG@OEFKCPOD@EGL_MAX_PBUFFER_WIDTH?$AA@ 000112f8     eglinfo.obj
 0001:00000310       ??_C@_09FJMIHJCN@EGL_LEVEL?$AA@ 00011310     eglinfo.obj
 0001:0000031c       ??_C@_0P@NOHGKAIH@EGL_DEPTH_SIZE?$AA@ 0001131c     eglinfo.obj
 0001:0000032c       ??_C@_0P@JBFIIOJI@EGL_CONFORMANT?$AA@ 0001132c     eglinfo.obj
 0001:0000033c       ??_C@_0BC@PJCLODMB@EGL_CONFIG_CAVEAT?$AA@ 0001133c     eglinfo.obj
 0001:00000350       ??_C@_0BG@NNCFGBKA@EGL_COLOR_BUFFER_TYPE?$AA@ 00011350     eglinfo.obj
 0001:00000368       ??_C@_0BJ@JNPDGLJA@EGL_BIND_TO_TEXTURE_RGBA?$AA@ 00011368     eglinfo.obj
 0001:00000384       ??_C@_0BI@CAMHEOID@EGL_BIND_TO_TEXTURE_RGB?$AA@ 00011384     eglinfo.obj
 0001:0000039c       ??_C@_0BE@PLMIBNKA@EGL_ALPHA_MASK_SIZE?$AA@ 0001139c     eglinfo.obj
 0001:000003b0       ??_C@_0P@ONLIEGLI@EGL_ALPHA_SIZE?$AA@ 000113b0     eglinfo.obj
 0001:000003c0       ??_C@_0BD@CCJDJFLK@EGL_LUMINANCE_SIZE?$AA@ 000113c0     eglinfo.obj
 0001:000003d4       ??_C@_0O@NEMBNDJO@EGL_BLUE_SIZE?$AA@ 000113d4     eglinfo.obj
 0001:000003e4       ??_C@_0P@LHHAFPKG@EGL_GREEN_SIZE?$AA@ 000113e4     eglinfo.obj
 0001:000003f4       ??_C@_0N@IFFAGPOM@EGL_RED_SIZE?$AA@ 000113f4     eglinfo.obj
 0001:00000404       ??_C@_0BA@OFNHAGGF@EGL_BUFFER_SIZE?$AA@ 00011404     eglinfo.obj
 0001:00000414       ??_C@_0O@CAFBEHGK@EGL_CONFIG_ID?$AA@ 00011414     eglinfo.obj
 0001:00000424       ??_C@_0BB@BCECMJFP@EGL_CONTEXT_LOST?$AA@ 00011424     eglinfo.obj
 0001:00000438       ??_C@_0BG@JCAPPMPM@EGL_BAD_NATIVE_WINDOW?$AA@ 00011438     eglinfo.obj
 0001:00000450       ??_C@_0BG@IANPFEBH@EGL_BAD_NATIVE_PIXMAP?$AA@ 00011450     eglinfo.obj
 0001:00000468       ??_C@_0BC@OMABNJPB@EGL_BAD_PARAMETER?$AA@ 00011468     eglinfo.obj
 0001:0000047c       ??_C@_0O@GCFMIHO@EGL_BAD_MATCH?$AA@ 0001147c     eglinfo.obj
 0001:0000048c       ??_C@_0BA@ECMACICF@EGL_BAD_SURFACE?$AA@ 0001148c     eglinfo.obj
 0001:0000049c       ??_C@_0BA@KHKFAGME@EGL_BAD_DISPLAY?$AA@ 0001149c     eglinfo.obj
 0001:000004ac       ??_C@_0BI@KBFIGPCO@EGL_BAD_CURRENT_SURFACE?$AA@ 000114ac     eglinfo.obj
 0001:000004c4       ??_C@_0BA@FPCJCEFK@EGL_BAD_CONTEXT?$AA@ 000114c4     eglinfo.obj
 0001:000004d4       ??_C@_0P@HOPKKPDK@EGL_BAD_CONFIG?$AA@ 000114d4     eglinfo.obj
 0001:000004e4       ??_C@_0BC@NLAJAPHP@EGL_BAD_ATTRIBUTE?$AA@ 000114e4     eglinfo.obj
 0001:000004f8       ??_C@_0O@PGDEJDGL@EGL_BAD_ALLOC?$AA@ 000114f8     eglinfo.obj
 0001:00000508       ??_C@_0P@ELJNOEME@EGL_BAD_ACCESS?$AA@ 00011508     eglinfo.obj
 0001:00000518       ??_C@_0BE@JIJLFFAN@EGL_NOT_INITIALIZED?$AA@ 00011518     eglinfo.obj
 0001:0000052c       ??_C@_0M@JFIJMCIK@EGL_SUCCESS?$AA@ 0001152c     eglinfo.obj
 0001:00000710       ??_C@_0BI@KDGOMBAC@?5egl?5error?5?8?$CFs?8?5?$CI0x?$CFx?$CJ?6?$AA@ 00011710     eglinfo.obj
 0001:00000728       ??_C@_0BP@HLDIKGBL@Unable?5to?5make?5current?5context?$AA@ 00011728     eglinfo.obj
 0001:00000748       ??_C@_0BO@OFBGKELB@Failed?5to?5get?5context?5attrib?6?$AA@ 00011748     eglinfo.obj
 0001:00000768       ??_C@_0BK@DPEOOONH@?6EGL?5context?5Attributes?3?6?$AA@ 00011768     eglinfo.obj
 0001:00000784       ??_C@_0BM@DDPOGPLK@Unable?5to?5create?5a?5context?6?$AA@ 00011784     eglinfo.obj
 0001:000007a0       ??_C@_0BN@MJJKBPIG@Failed?5to?5get?5surface?5attrib?$AA@ 000117a0     eglinfo.obj
 0001:000007c0       ??_C@_0M@NPBDCADI@?5?$CFs?5?$DN?50x?$CFx?6?$AA@ 000117c0     eglinfo.obj
 0001:000007cc       ??_C@_0BK@CJOIJNJN@?6EGL?5surface?5Attributes?3?6?$AA@ 000117cc     eglinfo.obj
 0001:000007e8       ??_C@_0CB@LFKEDNNA@Unable?5to?5create?5pbuffer?5surface@ 000117e8     eglinfo.obj
 0001:0000080c       ??_C@_0CA@NOEBEKGP@Unable?5to?5create?5window?5surface?$AA@ 0001180c     eglinfo.obj
 0001:0000082c       ??_C@_0BM@JMLGKGPI@Failed?5to?5get?5config?5attrib?$AA@ 0001182c     eglinfo.obj
 0001:00000848       ??_C@_01EEMJAFIK@?6?$AA@   00011848     eglinfo.obj
 0001:0000084c       ??_C@_0BE@OOAKOGAL@?5EGL_OPENGL_ES_BIT?5?$AA@ 0001184c     eglinfo.obj
 0001:00000860       ??_C@_0BB@NJHBLDLL@?5EGL_OPENVG_BIT?5?$AA@ 00011860     eglinfo.obj
 0001:00000874       ??_C@_0BF@NBMKLFHD@?5EGL_OPENGL_ES2_BIT?5?$AA@ 00011874     eglinfo.obj
 0001:0000088c       ??_C@_0BN@ODBDDGHG@?5EGL_VG_ALPHA_FORMAT_PRE_BIT?$AA@ 0001188c     eglinfo.obj
 0001:000008ac       ??_C@_0BP@IPGHOKOG@?5EGL_VG_COLORSPACE_LINEAR_BIT?5?$AA@ 000118ac     eglinfo.obj
 0001:000008cc       ??_C@_0BB@GPDKBFFA@?5EGL_WINDOW_BIT?5?$AA@ 000118cc     eglinfo.obj
 0001:000008e0       ??_C@_0BB@ENJMJHJH@?5EGL_PIXMAP_BIT?5?$AA@ 000118e0     eglinfo.obj
 0001:000008f4       ??_C@_0BC@LBLKPAPA@?5EGL_PBUFFER_BIT?5?$AA@ 000118f4     eglinfo.obj
 0001:00000908       ??_C@_0M@LAHIOMBA@?5?$CFs?5?$DN?50x?$CFx?5?$AA@ 00011908     eglinfo.obj
 0001:00000914       ??_C@_0CF@HADODIPA@?6?$CK?$CK?$CK?$CK?$CK?$CK?$CK?$CK?$CK?$CK?$CK?$CK?$CK?$CK?$CK?$CK?$CK?$CK?$CK?$CK?$CK?$CK?$CK?$CK?$CK?$CK?$CK?$CK?$CK?$CK?$CK@ 00011914     eglinfo.obj
 0001:0000093c       ??_C@_0BD@ELPCDIKM@EGL?5Config?5num?5?$CFu?6?$AA@ 0001193c     eglinfo.obj
 0001:00000950       ??_C@_0BH@DJNHOJJI@EGL?5vendor?5string?3?5?$CFs?6?$AA@ 00011950     eglinfo.obj
 0001:00000968       ??_C@_0BI@HBKAJDDC@EGL?5version?5string?3?5?$CFs?6?$AA@ 00011968     eglinfo.obj
 0001:00000980       ??_C@_0BE@EEJFKDHF@EGL?5extensions?3?5?$CFs?6?$AA@ 00011980     eglinfo.obj
 0001:00000994       ??_C@_0BJ@PJOLGCLH@EGL?5client?5APIs?5are?3?5?$CFs?6?$AA@ 00011994     eglinfo.obj
 0001:000009b0       ??_C@_0BJ@JBOLJEME@?6EGL?5config?5Attributes?3?6?$AA@ 000119b0     eglinfo.obj
 0001:000009cc       ??_C@_0DA@PMCIHGDE@?6?$CK?$CK?$CK?$CK?$CK?$CK?$CK?$CK?$CK?$CK?$CK?$CK?$CK?$CK?$CK?$CK?$CK?$CK?$CK?$CK?$CK?$CK?$CK?$CK?$CK?$CK?$CK?$CK?$CK?$CK?$CK@ 000119cc     eglinfo.obj
 0001:000009fc       ??_C@_0BH@FDCEEPEG@?6OpenGL?5Information?3?5?6?$AA@ 000119fc     eglinfo.obj
 0001:00000a14       ??_C@_0CJ@GAAECDFN@Unable?5to?5make?5current?5an?5OpenGL@ 00011a14     eglinfo.obj
 0001:00000a40       ??_C@_0CE@CBMNDBFP@Unable?5to?5create?5an?5OpenGL?5conte@ 00011a40     eglinfo.obj
 0001:00000a64       ??_C@_0BM@HJBOIKD@?6OpenGL_ES?51?5Information?3?5?6?$AA@ 00011a64     eglinfo.obj
 0001:00000a80       ??_C@_0BM@FEALLDCH@?6OpenGL_ES?52?5Information?3?5?6?$AA@ 00011a80     eglinfo.obj
 0001:00000a9c       ??_C@_0BH@CHFPLBKF@?6OpenVG?5Information?3?5?6?$AA@ 00011a9c     eglinfo.obj
 0001:00000ab4       ??_C@_0BG@LGDLAGIF@Failed?5to?5get?5configs?$AA@ 00011ab4     eglinfo.obj
 0001:00000acc       ??_C@_0BL@BEAIAHEF@Failed?5to?5get?5config?5count?$AA@ 00011acc     eglinfo.obj
 0001:00000ae8       ??_C@_0BJ@IGFEHMHO@Unable?5to?5initialise?5egl?$AA@ 00011ae8     eglinfo.obj
 0001:00000b04       ??_C@_0BK@HMFIJNFM@Unable?5to?5get?5egl?5display?$AA@ 00011b04     eglinfo.obj
 0001:00000b20       ??_C@_0CN@GDPGAION@Usage?3?5eglinfo?5?$FLh?$FN?5?$FL?9a?$FN?5?$FL?9e?$FN?5?$FL?9v@ 00011b20     eglinfo.obj
 0001:00000b50       ??_C@_0N@MBOKGNDP@?7?9h?3?5Help?4?5?6?$AA@ 00011b50     eglinfo.obj
 0001:00000b60       ??_C@_0FB@PFPFNFBN@?7?9a?3?5Print?5all?5the?5possible?5EGL?0@ 00011b60     eglinfo.obj
 0001:00000bb4       ??_C@_0BL@PINDPDPK@?7?9e?3?5Print?5only?5EGL?5info?4?6?$AA@ 00011bb4     eglinfo.obj
 0001:00000bd0       ??_C@_0BO@OLGJBEHN@?7?9v?3?5Print?5only?5OpenVG?5info?4?6?$AA@ 00011bd0     eglinfo.obj
 0001:00000bf0       ??_C@_0BO@LLLKEMLL@?7?9g?3?5Print?5only?5OpenGL?5info?4?6?$AA@ 00011bf0     eglinfo.obj
 0001:00000c10       ??_C@_0CD@DANHAADO@?7?91?3?5Print?5only?5OpenGL?5ES?51?5info@ 00011c10     eglinfo.obj
 0001:00000c34       ??_C@_0CD@FCENINOO@?7?92?3?5Print?5only?5OpenGL?5ES?52?5info@ 00011c34     eglinfo.obj
 0001:00000c58       ??_C@_0BF@CIBJNFIB@Unknown?5option?5?$GA?$CFs?8?6?$AA@ 00011c58     eglinfo.obj
 0001:00000c70       ??_C@_02JNAPBCPB@?9h?$AA@  00011c70     eglinfo.obj
 0001:00000c74       ??_C@_02NNFLKHCP@?92?$AA@  00011c74     eglinfo.obj
 0001:00000c78       ??_C@_02PGHGPEOM@?91?$AA@  00011c78     eglinfo.obj
 0001:00000c7c       ??_C@_02BKJHAODO@?9g?$AA@  00011c7c     eglinfo.obj
 0001:00000c80       ??_C@_02EJEOCNCO@?9v?$AA@  00011c80     eglinfo.obj
 0001:00000c84       ??_C@_02CIKBGMLM@?9e?$AA@  00011c84     eglinfo.obj
 0001:00000c88       ??_C@_02EMMNKJLI@?9a?$AA@  00011c88     eglinfo.obj
 0001:00000c8c       ??_C@_0BG@MHPLLPCH@Config?5index?5too?5high?$AA@ 00011c8c     eglinfo.obj
 0001:00000ca4       ??_C@_0BM@KKOHJEF@GL_ALIASED_LINE_WIDTH_RANGE?$AA@ 00011ca4     ex_gles2.obj
 0001:00000cc0       ??_C@_0BM@EOKMFJL@GL_ALIASED_POINT_SIZE_RANGE?$AA@ 00011cc0     ex_gles2.obj
 0001:00000cdc       ??_C@_0CE@FCBBJEFH@GL_IMPLEMENTATION_COLOR_READ_FOR@ 00011cdc     ex_gles2.obj
 0001:00000d00       ??_C@_0CC@PANPEJM@GL_IMPLEMENTATION_COLOR_READ_TYP@ 00011d00     ex_gles2.obj
 0001:00000d24       ??_C@_0BJ@OGPAIIDC@GL_MAX_RENDERBUFFER_SIZE?$AA@ 00011d24     ex_gles2.obj
 0001:00000d40       ??_C@_0CA@GDELLFP@GL_MAX_FRAGMENT_UNIFORM_VECTORS?$AA@ 00011d40     ex_gles2.obj
 0001:00000d60       ??_C@_0BL@MBFIJDNJ@GL_MAX_TEXTURE_IMAGE_UNITS?$AA@ 00011d60     ex_gles2.obj
 0001:00000d7c       ??_C@_0CC@DCGLGBBC@GL_MAX_VERTEX_TEXTURE_IMAGE_UNIT@ 00011d7c     ex_gles2.obj
 0001:00000da0       ??_C@_0CE@IJBMLCEP@GL_MAX_COMBINED_TEXTURE_IMAGE_UN@ 00011da0     ex_gles2.obj
 0001:00000dc4       ??_C@_0BH@JAAOIIAM@GL_MAX_VARYING_VECTORS?$AA@ 00011dc4     ex_gles2.obj
 0001:00000ddc       ??_C@_0BO@HAJDDPFB@GL_MAX_VERTEX_UNIFORM_VECTORS?$AA@ 00011ddc     ex_gles2.obj
 0001:00000dfc       ??_C@_0BG@CLFCOANJ@GL_MAX_VERTEX_ATTRIBS?$AA@ 00011dfc     ex_gles2.obj
 0001:00000e14       ??_C@_0BN@LCEKMJOA@GL_NUM_SHADER_BINARY_FORMATS?$AA@ 00011e14     ex_gles2.obj
 0001:00000e34       ??_C@_0CC@LGFBHBLD@GL_NUM_COMPRESSED_TEXTURE_FORMAT@ 00011e34     ex_gles2.obj
 0001:00000e58       ??_C@_0BF@BBCKGPMC@GL_MAX_VIEWPORT_DIMS?$AA@ 00011e58     ex_gles2.obj
 0001:00000e70       ??_C@_0BN@PMOODMBD@GL_MAX_CUBE_MAP_TEXTURE_SIZE?$AA@ 00011e70     ex_gles2.obj
 0001:00000e90       ??_C@_0BE@LGLBMFFL@GL_MAX_TEXTURE_SIZE?$AA@ 00011e90     ex_gles2.obj
 0001:00000ea4       ??_C@_0BB@HJIHLJMI@GL_SUBPIXEL_BITS?$AA@ 00011ea4     ex_gles2.obj
 0001:00000eb8       ??_C@_0BD@HPAPEICD@GL_DEPTH_WRITEMASK?$AA@ 00011eb8     ex_gles2.obj
 0001:00000ecc       ??_C@_0BD@BMFPHMOF@GL_COLOR_WRITEMASK?$AA@ 00011ecc     ex_gles2.obj
 0001:00000ee0       ??_C@_0BD@MJEBJGFO@GL_SHADER_COMPILER?$AA@ 00011ee0     ex_gles2.obj
 0001:00000ef4       ??_C@_0O@MDNPDBLF@GL_EXTENSIONS?$AA@ 00011ef4     ex_gles2.obj
 0001:00000f04       ??_C@_0BM@EPHGGKHF@GL_SHADING_LANGUAGE_VERSION?$AA@ 00011f04     ex_gles2.obj
 0001:00000f20       ??_C@_0L@KMJCIEP@GL_VERSION?$AA@ 00011f20     ex_gles2.obj
 0001:00000f2c       ??_C@_0M@OGHDLCMI@GL_RENDERER?$AA@ 00011f2c     ex_gles2.obj
 0001:00000f38       ??_C@_09MLNNABBC@GL_VENDOR?$AA@ 00011f38     ex_gles2.obj
 0001:00001070       ??_C@_04LGCOOLNK@?5?$CFf?5?$AA@ 00012070     ex_gles2.obj
 0001:00001078       ??_C@_0BN@DBKAJGMK@?6GLES?52?5Float?5Information?5?3?6?$AA@ 00012078     ex_gles2.obj
 0001:00001098       ??_C@_0M@CKCOBONE@glGetFloatv?$AA@ 00012098     ex_gles2.obj
 0001:000010a4       ??_C@_0BP@COMKKFE@?6GLES?52?5Integer?5Information?5?3?6?$AA@ 000120a4     ex_gles2.obj
 0001:000010c4       ??_C@_0O@DHHDCCLF@glGetIntegerv?$AA@ 000120c4     ex_gles2.obj
 0001:000010d4       ??_C@_06DIHMPHPI@?50x?$CFx?5?$AA@ 000120d4     ex_gles2.obj
 0001:000010dc       ??_C@_06FNDIOKNI@?5?$CFs?5?$DN?5?$AA@ 000120dc     ex_gles2.obj
 0001:000010e4       ??_C@_0BP@HDHJOANJ@?6GLES?52?5Boolean?5Information?5?3?6?$AA@ 000120e4     ex_gles2.obj
 0001:00001104       ??_C@_0O@NLMELLCJ@glGetBooleanv?$AA@ 00012104     ex_gles2.obj
 0001:00001114       ??_C@_0L@PHNJFENO@?5?$CFs?5?$DN?5?$CFs?5?6?$AA@ 00012114     ex_gles2.obj
 0001:00001120       ??_C@_0O@HFAAEHFL@libGLESv2?4dll?$AA@ 00012120     ex_gles2.obj
 0001:00001130       ??_C@_0BO@LABNBOAG@?6GLES?52?5String?5Information?5?3?6?$AA@ 00012130     ex_gles2.obj
 0001:00001150       ??_C@_0M@OPOBFDCB@glGetString?$AA@ 00012150     ex_gles2.obj
 0001:0000115c       ??_C@_0BL@IBBBELHI@GL_SMOOTH_LINE_WIDTH_RANGE?$AA@ 0001215c     ex_gles.obj
 0001:00001178       ??_C@_0BL@IPFFPHKG@GL_SMOOTH_POINT_SIZE_RANGE?$AA@ 00012178     ex_gles.obj
 0001:00001194       ??_C@_0BF@FGKIDJBF@GL_MAX_TEXTURE_UNITS?$AA@ 00012194     ex_gles.obj
 0001:000011ac       ??_C@_0BL@IBNHBMJE@GL_MAX_TEXTURE_STACK_DEPTH?$AA@ 000121ac     ex_gles.obj
 0001:000011c8       ??_C@_0BO@PDBIOMDD@GL_MAX_PROJECTION_STACK_DEPTH?$AA@ 000121c8     ex_gles.obj
 0001:000011e8       ??_C@_0BN@MMJNENIG@GL_MAX_MODELVIEW_STACK_DEPTH?$AA@ 000121e8     ex_gles.obj
 0001:00001208       ??_C@_0BD@MDDIOKKJ@GL_MAX_CLIP_PLANES?$AA@ 00012208     ex_gles.obj
 0001:0000121c       ??_C@_0O@KPGMDEIP@GL_MAX_LIGHTS?$AA@ 0001221c     ex_gles.obj
 0001:000012f8       ??_C@_0BL@DMKCDHKB@?6GLES?5Float?5Information?5?3?6?$AA@ 000122f8     ex_gles.obj
 0001:00001314       ??_C@_0BN@CFDEIGEE@?6GLES?5Integer?5Information?5?3?6?$AA@ 00012314     ex_gles.obj
 0001:00001334       ??_C@_0P@MADFBLIB@libGLES_CM?4dll?$AA@ 00012334     ex_gles.obj
 0001:00001344       ??_C@_0BM@GKHAKEHH@?6GLES?5String?5Information?5?3?6?$AA@ 00012344     ex_gles.obj
 0001:00001360       ??_C@_0CC@KODEIKLD@Successfully?5loaded?5library?5?$CFs?4?5@ 00012360     ex_wince.obj
 0001:00001384       ??_C@_0CG@IFGHKLBK@Couldn?8t?5load?5library?5?$CFs?3?5Error?5@ 00012384     ex_wince.obj
 0001:000013ac       ??_C@_0BH@HKOLHCFB@invalid?5library?5handle?$AA@ 000123ac     ex_wince.obj
 0001:000013c4       ??_C@_0CF@FNGBCMCJ@FreeLibrary?5failed?5to?5close?5libr@ 000123c4     ex_wince.obj
 0001:000013ec       ??_C@_0N@CPFAKHMA@VG_MAX_FLOAT?$AA@ 000123ec     ex_vg.obj
 0001:000013fc       ??_C@_0BO@HKAFEMJP@VG_MAX_GAUSSIAN_STD_DEVIATION?$AA@ 000123fc     ex_vg.obj
 0001:0000141c       ??_C@_0BD@EEINCNLK@VG_MAX_IMAGE_BYTES?$AA@ 0001241c     ex_vg.obj
 0001:00001430       ??_C@_0BE@JLHLFPBI@VG_MAX_IMAGE_PIXELS?$AA@ 00012430     ex_vg.obj
 0001:00001444       ??_C@_0BE@HEJAFGI@VG_MAX_IMAGE_HEIGHT?$AA@ 00012444     ex_vg.obj
 0001:00001458       ??_C@_0BD@JDLNHMFC@VG_MAX_IMAGE_WIDTH?$AA@ 00012458     ex_vg.obj
 0001:0000146c       ??_C@_0BI@NGLLIMNO@VG_MAX_COLOR_RAMP_STOPS?$AA@ 0001246c     ex_vg.obj
 0001:00001484       ??_C@_0BN@GGLNPIHE@VG_MAX_SEPARABLE_KERNEL_SIZE?$AA@ 00012484     ex_vg.obj
 0001:000014a4       ??_C@_0BD@HIBAIPLP@VG_MAX_KERNEL_SIZE?$AA@ 000124a4     ex_vg.obj
 0001:000014b8       ??_C@_0BC@LGEIGDCP@VG_MAX_DASH_COUNT?$AA@ 000124b8     ex_vg.obj
 0001:000014cc       ??_C@_0BF@OIMNPOIM@VG_MAX_SCISSOR_RECTS?$AA@ 000124cc     ex_vg.obj
 0001:000014e4       ??_C@_0O@NPKLFDAM@VG_EXTENSIONS?$AA@ 000124e4     ex_vg.obj
 0001:000014f4       ??_C@_0L@JNFBMILD@VG_VERSION?$AA@ 000124f4     ex_vg.obj
 0001:00001500       ??_C@_0M@FCOPJEBP@VG_RENDERER?$AA@ 00012500     ex_vg.obj
 0001:0000150c       ??_C@_09IBOEHFBJ@VG_VENDOR?$AA@ 0001250c     ex_vg.obj
 0001:00001590       ??_C@_0CH@IKLIOHGM@?6VG?5API?5Float?5Parameter?5Informat@ 00012590     ex_vg.obj
 0001:000015b8       ??_C@_06HOKOHFLH@vgGetf?$AA@ 000125b8     ex_vg.obj
 0001:000015c0       ??_C@_0L@CCJJPDKD@?5?$CFs?5?$DN?5?$CFE?5?6?$AA@ 000125c0     ex_vg.obj
 0001:000015cc       ??_C@_0N@OHOIIAAC@?5?$CFs?5?$DN?50x?$CFx?5?6?$AA@ 000125cc     ex_vg.obj
 0001:000015dc       ??_C@_0BL@NAOKPPOP@?6VG?5Integer?5Information?5?3?6?$AA@ 000125dc     ex_vg.obj
 0001:000015f8       ??_C@_06PJDGGJHI@vgGeti?$AA@ 000125f8     ex_vg.obj
 0001:00001600       ??_C@_0O@LFGHKFEJ@libOpenVG?4dll?$AA@ 00012600     ex_vg.obj
 0001:00001610       ??_C@_0BO@IKFKCEGL@?6VG?5API?5String?5Information?5?3?6?$AA@ 00012610     ex_vg.obj
 0001:00001630       ??_C@_0M@FLHNHFPG@vgGetString?$AA@ 00012630     ex_vg.obj
 0001:00001708       ??_C@_0BJ@LCCLPBAE@?6GL?5Float?5Information?5?3?6?$AA@ 00012708     ex_gl.obj
 0001:00001724       ??_C@_0BL@IEEDCHOE@?6GL?5Integer?5Information?5?3?6?$AA@ 00012724     ex_gl.obj
 0001:00001740       ??_C@_0N@DOKAJOHF@opengl32?4dll?$AA@ 00012740     ex_gl.obj
 0001:00001750       ??_C@_0BK@MMECHKNG@?6GL?5String?5Information?5?3?6?$AA@ 00012750     ex_gl.obj
 0001:00001770       ??_C@_1KE@BDGMONOJ@?$AAH?$AA?3?$AA?2?$AAW?$AAI?$AAN?$AAC?$AAE?$AA6?$AA0?$AA0?$AA?2?$AAP?$AAL?$AAA?$AAT?$AAF?$AAO?$AAR?$AAM?$AA?2?$AAS?$AAM?$AAD?$AAK?$AAV?$AA2?$AA1?$AA0?$AA?2?$AAS?$AAR@ 00012770     wince_unittests.obj
 0001:00001814       ??_C@_1CI@OHCJFJPM@?$AAE?$AAR?$AAR?$AAO?$AAR?$AA?3?$AA?5?$AA?$CF?$AAs?$AA?5?$AAl?$AAi?$AAn?$AAe?$AA?5?$AA?$CF?$AAd?$AA?3?$AA?5?$AA?$AA@ 00012814     wince_unittests.obj
 0001:0000183c       ??_C@_1CK@MPGKAOE@?$AA?$CI?$AAe?$AAr?$AAr?$AAo?$AAr?$AA?5?$AAc?$AAo?$AAd?$AAe?$AA?3?$AA?5?$AA?$CF?$AAd?$AA?$CJ?$AA?3?$AA?5?$AA?$CF?$AAs?$AA?$AA@ 0001283c     wince_unittests.obj
 0001:00001868       ??_C@_1M@DMCDIEDK@?$AAP?$AAK?$AAM?$AA1?$AA?3?$AA?$AA@ 00012868     wince_unittests.obj
 0001:00001874       ??_C@_0L@GPAGIAIC@?9disablepm?$AA@ 00012874     wince_unittests.obj
 0001:00001880       ??_C@_07FBLHGNAH@app?4exe?$AA@ 00012880     wince_unittests.obj
 0001:00002c5c       ProcessOptions             00013c5c f   eglinfo.obj
 0001:00002db0       main                       00013db0 f   eglinfo.obj
 0001:00002f7c       PrintOnlyOpenGLES2Info     00013f7c f   ex_gles2.obj
 0001:000031e0       PrintOnlyOpenGLESInfo      000141e0 f   ex_gles.obj
 0001:000033bc       exLoadLibrary              000143bc f   ex_wince.obj
 0001:00003450       exUnloadLibrary            00014450 f   ex_wince.obj
 0001:00003494       exGetLibFuncAddr           00014494 f   ex_wince.obj
 0001:0000351c       PrintOnlyOpenVGInfo        0001451c f   ex_vg.obj
 0001:0000365c       PrintOnlyOpenGLInfo        0001465c f   ex_gl.obj
 0001:00003830       WinMain                    00014830 f   wince_unittests.obj
 0001:00003a58       GetLastError               00014a58 f   coredll:COREDLL.dll
 0001:00003a68       LoadLibraryW               00014a68 f   coredll:COREDLL.dll
 0001:00003a78       FreeLibrary                00014a78 f   coredll:COREDLL.dll
 0001:00003a88       GetProcAddressW            00014a88 f   coredll:COREDLL.dll
 0001:00003a98       ReleasePowerRequirement    00014a98 f   coredll:COREDLL.dll
 0001:00003aa8       NKDbgPrintfW               00014aa8 f   coredll:COREDLL.dll
 0001:00003ab8       FormatMessageW             00014ab8 f   coredll:COREDLL.dll
 0001:00003ac8       SetPowerRequirement        00014ac8 f   coredll:COREDLL.dll
 0001:00003ad8       WideCharToMultiByte        00014ad8 f   coredll:COREDLL.dll
 0001:00003b68       WinMainCRTStartup          00014b68 f   corelib0:pegwmain.obj
 0001:00003b9c       __GSHandlerCheckCommon     00014b9c f   corelib0:gshandler.obj
 0001:00003bd8       __GSHandlerCheck           00014bd8 f   corelib0:gshandler.obj
 0001:00003bfc       __security_init_cookie     00014bfc f   corelib0:seccinit.obj
 0001:00003c58       __security_check_cookie    00014c58 f   corelib0:armsecgs.obj
 0001:00003c6c       __gsfailure                00014c6c f   corelib0:armsecgs.obj
 0001:00003d78       exit                       00014d78 f   corelib0:cexit.obj
 0001:00003d90       _exit                      00014d90 f   corelib0:cexit.obj
 0001:00003dd0       _initterm                  00014dd0 f   corelib0:crt0dat.obj
 0001:00003e04       _cinit                     00014e04 f   corelib0:crt0dat.obj
 0001:00003e38       fprintf                    00014e38 f   corelib1:COREDLL.dll
 0001:00003e48       _getstdfilex               00014e48 f   corelib1:COREDLL.dll
 0001:00003e58       printf                     00014e58 f   corelib1:COREDLL.dll
 0001:00003e68       free                       00014e68 f   corelib1:COREDLL.dll
 0001:00003e78       malloc                     00014e78 f   corelib1:COREDLL.dll
 0001:00003e88       strcmp                     00014e88 f   corelib1:COREDLL.dll
 0001:00003e98       mbstowcs                   00014e98 f   corelib1:COREDLL.dll
 0001:00003ea8       strlen                     00014ea8 f   corelib1:COREDLL.dll
 0001:00003eb8       memset                     00014eb8 f   corelib1:COREDLL.dll
 0001:00003ec8       _stricmp                   00014ec8 f   corelib1:COREDLL.dll
 0001:00003ed8       _isctype                   00014ed8 f   corelib1:COREDLL.dll
 0001:00003ee8       wcslen                     00014ee8 f   corelib1:COREDLL.dll
 0001:00003ef8       _XcptFilter                00014ef8 f   corelib1:COREDLL.dll
 0001:00003f08       __C_specific_handler       00014f08 f   corelib1:COREDLL.dll
 0001:00003f18       __security_gen_cookie2     00014f18 f   corelib1:COREDLL.dll
 0001:00003f28       __report_gsfailure         00014f28 f   corelib1:COREDLL.dll
 0001:00003f38       TerminateProcess           00014f38 f   coredll:COREDLL.dll
 0001:00003f64       __IMPORT_DESCRIPTOR_libEGL 00014f64     libEGL:libEGL.dll
 0001:00003f78       __IMPORT_DESCRIPTOR_COREDLL 00014f78     coredll:COREDLL.dll
 0001:00003f8c       __NULL_IMPORT_DESCRIPTOR   00014f8c     libEGL:libEGL.dll
 0002:00000000       __imp_FormatMessageW       00016000     coredll:COREDLL.dll
 0002:00000004       __imp___report_gsfailure   00016004     corelib1:COREDLL.dll
 0002:00000008       __imp___security_gen_cookie2 00016008     corelib1:COREDLL.dll
 0002:0000000c       __imp___C_specific_handler 0001600c     corelib1:COREDLL.dll
 0002:00000010       __imp__XcptFilter          00016010     corelib1:COREDLL.dll
 0002:00000014       __imp_wcslen               00016014     corelib1:COREDLL.dll
 0002:00000018       __imp__isctype             00016018     corelib1:COREDLL.dll
 0002:0000001c       __imp__stricmp             0001601c     corelib1:COREDLL.dll
 0002:00000020       __imp_memset               00016020     corelib1:COREDLL.dll
 0002:00000024       __imp_strlen               00016024     corelib1:COREDLL.dll
 0002:00000028       __imp_mbstowcs             00016028     corelib1:COREDLL.dll
 0002:0000002c       __imp___stod               0001602c     corelib1:COREDLL.dll
 0002:00000030       __imp_strcmp               00016030     corelib1:COREDLL.dll
 0002:00000034       __imp_malloc               00016034     corelib1:COREDLL.dll
 0002:00000038       __imp_free                 00016038     corelib1:COREDLL.dll
 0002:0000003c       __imp_GetLastError         0001603c     coredll:COREDLL.dll
 0002:00000040       __imp_LoadLibraryW         00016040     coredll:COREDLL.dll
 0002:00000044       __imp_FreeLibrary          00016044     coredll:COREDLL.dll
 0002:00000048       __imp_GetProcAddressW      00016048     coredll:COREDLL.dll
 0002:0000004c       __imp_ReleasePowerRequirement 0001604c     coredll:COREDLL.dll
 0002:00000050       __imp_NKDbgPrintfW         00016050     coredll:COREDLL.dll
 0002:00000054       __imp_TerminateProcess     00016054     coredll:COREDLL.dll
 0002:00000058       __imp_SetPowerRequirement  00016058     coredll:COREDLL.dll
 0002:0000005c       __imp_WideCharToMultiByte  0001605c     coredll:COREDLL.dll
 0002:00000060       __imp_fprintf              00016060     corelib1:COREDLL.dll
 0002:00000064       __imp__getstdfilex         00016064     corelib1:COREDLL.dll
 0002:00000068       __imp_printf               00016068     corelib1:COREDLL.dll
 0002:0000006c       \177COREDLL_NULL_THUNK_DATA 0001606c     coredll:COREDLL.dll
 0002:00000070       __imp_eglTerminate         00016070     libEGL:libEGL.dll
 0002:00000074       __imp_eglGetDisplay        00016074     libEGL:libEGL.dll
 0002:00000078       __imp_eglInitialize        00016078     libEGL:libEGL.dll
 0002:0000007c       __imp_eglGetConfigs        0001607c     libEGL:libEGL.dll
 0002:00000080       __imp_eglQueryString       00016080     libEGL:libEGL.dll
 0002:00000084       __imp_eglGetConfigAttrib   00016084     libEGL:libEGL.dll
 0002:00000088       __imp_eglGetError          00016088     libEGL:libEGL.dll
 0002:0000008c       __imp_eglCreateWindowSurface 0001608c     libEGL:libEGL.dll
 0002:00000090       __imp_eglCreatePbufferSurface 00016090     libEGL:libEGL.dll
 0002:00000094       __imp_eglQuerySurface      00016094     libEGL:libEGL.dll
 0002:00000098       __imp_eglCreateContext     00016098     libEGL:libEGL.dll
 0002:0000009c       __imp_eglBindAPI           0001609c     libEGL:libEGL.dll
 0002:000000a0       __imp_eglQueryContext      000160a0     libEGL:libEGL.dll
 0002:000000a4       __imp_eglMakeCurrent       000160a4     libEGL:libEGL.dll
 0002:000000a8       __imp_eglDestroySurface    000160a8     libEGL:libEGL.dll
 0002:000000ac       __imp_eglDestroyContext    000160ac     libEGL:libEGL.dll
 0002:000000b0       \177libEGL_NULL_THUNK_DATA 000160b0     libEGL:libEGL.dll
 0002:000000b4       __security_cookie          000160b4     corelib0:seccinit.obj
 0002:000000b8       __security_cookie_complement 000160b8     corelib0:seccinit.obj
 0002:000000cc       pfnRegisteredWndProc       000160cc     wince_unittests.obj
 0002:000000d0       _exitflag                  000160d0     corelib0:cexit.obj
 0002:000000d4       __onexitend                000160d4     <common>
 0002:000000d8       __onexitbegin              000160d8     <common>

 entry point at        0001:00003b68

 Static symbols

 0001:000018ac       handle_egl_error           000128ac f   eglinfo.obj
 0001:000018e4       PrintEGLInfo               000128e4 f   eglinfo.obj
 0001:00001f30       PrintGLInfo                00012f30 f   eglinfo.obj
 0001:000021cc       PrintGLES1Info             000131cc f   eglinfo.obj
 0001:0000248c       PrintGLES2Info             0001348c f   eglinfo.obj
 0001:0000274c       PrintVGInfo                0001374c f   eglinfo.obj
 0001:000029e8       EnumerateInfo              000139e8 f   eglinfo.obj
 0001:00003af0       WinMainCRTStartupHelper    00014af0 f   corelib0:pegwmain.obj
 0001:00003cb0       doexit                     00014cb0 f   corelib0:cexit.obj
